:10000000FC7F002015060000050600000906000020
:1000100000000000000000000000000000000000E0
:100020000000000000000000000000000D060000BD
:10003000000000000000000011060000650700003D
:1000400010B5064C2378002B07D1054B002B02D0AE
:10005000044800E000BF0123237010BD5C000020B5
:10006000000000000819000008B5084B002B03D061
:100070000748084900E000BF07480368002B03D089
:10008000064B002B00D0984708BDC046000000007A
:100090000819000060000020580000200000000047
:1000A000154A164B1178002909D115491878097895
:1000B0004118C9B21970802012498002C8611178B4
:1000C0000131C9B211701978F02902D819780929BB
:1000D00009D80B4908784042C0B2087018780978EE
:1000E0004118C9B2197012781B789A4203D1802244
:1000F000044B9202DA617047780000200100002072
:10010000000000200044004110B5C3699C07FCD4E6
:1001100003680224A3430360C46901231C42FBD18A
:100120000468234303600368DC07FCD4C46901232B
:100130001C42FBD1C469DC401C42F7D1084B1A4376
:100140000260C3695A07FCD4C0239B0243608181CB
:10015000C3699C07FCD4036802221343036010BDEB
:1001600004000040037EDA07FCD5018570470000DB
:10017000027E01235107FBD5428B1A4207D1428BE5
:10018000DA401A4203D1428B92081A4202D0034B42
:1001900001221A70008DC0B27047C046790000205D
:1001A00070B50368041C988B1A1C0821FF320842A2
:1001B00026D0802099839872112353704021144BCC
:1001C000917150715E68134DC0202E40800506432A
:1001D0005E605E693540284358610F4818600F48DB
:1001E00018615D680E4828408025AD02284358609C
:1001F0005868800B8003586000235171237105E01B
:10020000137ADA0602D5201C00F0E6FA207970BDD8
:1002100098010020FFFFFF8F9800002018010020A8
:10022000FF3F00F0002303714371044B01608360C2
:100230000B78022213430B707047C046A1010000E7
:1002400038B5364B2021DA6901200A43DA61344B94
:1002500006241A7802431A70324B0F221978914300
:1002600019701978214319702F490C7820430870B0
:1002700019780A401A701A7860210A431A702B4BB9
:100280002B4A5A805A7852B2002AFBDB294B0121B3
:100290001A780A431A709A78D107FCD42648026863
:1002A000510B1F221140914200D1052111408C01B8
:1002B0001D8D22492940214319850468A10C0A405B
:1002C0001F2A00D11D221C8D1F210A408C4322436E
:1002D0001A8502680721D20D0A408A4200D1032202
:1002E0000A40188D1103164A02400A431A851978EC
:1002F0007F220A401A701A78042112480A431A70A1
:1003000058621A890C218A431A811A8901218A4369
:100310001A810021802201F076F938BD00040040E6
:10032000584400413C44004159440041000C004005
:100330000640000000500041246080003FF8FFFFAD
:10034000FF8FFFFF98010020F7B5141C1F4A5F01C3
:1003500001971D1CD319061C5869271C4000400F2B
:1003600003301033C74006D00F1C80225968120694
:100370000A435A6009E02F1C7B1E9F41144BBF01AA
:10038000FF18381C221C01F035F901990F48083577
:1003900042181761131C5269A104920B890C920335
:1003A0000A435A6159690B4A0A405A616B01F318B2
:1003B0000222DA715979802252420A435A716B0142
:1003C000F318DB799A07FAD5201CFEBD98010020AE
:1003D00018010020FF3F00F0F8B51A4E051C3378D5
:1003E000141C002B12D1184B184A1A645A6C920B29
:1003F00092035A64586C164A02405A64A2235B0066
:10040000EA5C40200243EA54012333704827FF3757
:10041000EA5D0123134012D00B4B5A6C9204920CEC
:10042000A24202D25C6CA404A40C081C221C074942
:1004300001F0E0F80123EB550023337000E01C1CB1
:10044000201CF8BD7A00002098010020D800002070
:10045000FF3F00F0FF3083792022002900D11022D5
:100460001343837170470000084BFF305A69920BA9
:1004700092035A6102230372827980235B42134301
:100480008371037A9A07FCD57047C0469801002013
:1004900080235B421943C9B28172704770B5A023B3
:1004A00003225B00C254134B134A5C6CC0211440FE
:1004B00089050C4346255C64FF35402444550F4DA7
:1004C00030261D6490256D0046555D6B154029430F
:1004D000922559636D0080214155094D1D63B0255A
:1004E0006D0044555C6F22405A67B2235B00C154D3
:1004F00070BDC04698010020FFFFFF8FD80000208C
:100500005801002030B5364A1E235168082099430F
:1005100002231943516033498A6902438A61324890
:10052000324A9082908A03439382D3689807FCD51D
:100530002F4B012018701878C40704D52C48407838
:1005400040B20028F7DB01209860587840B20028BC
:10055000FBDB284C26484460587840B20028FBDB7F
:1005600082242348E4014480587840B20028FBDB11
:10057000908C8024A0439084D068C506FCD51E4C86
:100580001A48C462D4681948E506FBD5848C1B4D13
:100590002C438484D4681548E506FBD5848C022559
:1005A0002C438484D0680406FCD51048C0684506F6
:1005B000F8D5D068C406FCD500229A605A7852B2A9
:1005C000002AFBDB0E480A4A50605A7852B2002AD1
:1005D000FBDB00230B724B728B72CB7230BDC046BB
:1005E00000400041000400400C06000000080040EC
:1005F000000C004001050100B805FF7D040A000061
:10060000000703000EBEFEE70DBEFEE705BEFEE7D7
:1006100002BEFEE70E4A0F4838B5824204D10E4AA8
:100620000E4B93420ED10AE00D4C9442F7D00023BA
:10063000D1188842F3D9E55804330D60F8E700F08B
:1006400011F804E09342FAD2002102C3FAE7FEE770
:10065000000000205C000020A40300205C000020BB
:100660000C190000334A38B51368141C01331ED02E
:10067000D1B200291BD1304B1878012318402F4BE1
:100680000AD11D682E498D4201D118600FE0196012
:100690002C4901390029FCD11960236883F30888AB
:1006A000FF239A43284B9A60224B5B681847FFF759
:1006B00029FF62B600F0CCFD00F05AF8234B8022EF
:1006C000920223499A6008220A602249041C0A60A7
:1006D000802212059A609A611F4B204AC0215A60FD
:1006E000194A0906106A0002000A01431162002239
:1006F0009A6007221A60A368201C9847184B0028AC
:1007000001D001221A701A78002A05D0002000F0CA
:1007100093FA00F019FBFCE71B78002BEBD100F0FB
:100720000BFE0028E7D0012000F086FA00F00CFB59
:10073000FCE7C0460020000038040040FC7F002099
:100740003581730748E8010000ED00E000440041F6
:10075000884400419844004110E000E0E7030000B5
:100760007B00002008B5FFF79BFC00F0C9FA08BD2C
:1007700010B5054B054C2360FFF762FD201C216876
:10078000FFF750FD201C10BD005000411802002052
:1007900070B5051CC0B0081C161C0C1C00F03BFFFB
:1007A00040006A460323023053701070760801231C
:1007B000E218013A11785A00002906D1281C69462E
:1007C0000023FFF7C1FD40B070BDB342F6DA6846C2
:1007D00081520133ECE70000F7B5BA4A0468137898
:1007E000B949271CFF37051C102038720B7053784D
:1007F000B648B74E037093783380D17833880902B6
:100800000B4333801179B34B198051791888090251
:10081000084318809079B0490880D279088812027C
:1008200002430A8040227A71A84F3A78A64F1202FA
:1008300038780F1C0243A9488446181C624500D131
:10084000C2E020DC802149008A4200D16EE109DC4F
:10085000812A00D192E0822A00D195E0802A00D03E
:1008600064E18BE081235B009A4200D1CFE000DAA3
:1008700058E1C0239B009A4200D157E1984B9A421D
:1008800000D14FE152E190231B019A4269D015DC5F
:10089000D023DB009A4222D088231B019A4269D0E0
:1008A000A023DB009A4200D040E1201CFFF7DCFDD2
:1008B0003188286889B2FFF7EBFD3BE1894B9A420A
:1008C00000D12FE100DC31E1874B9A4200D11DE1DC
:1008D000864B9A4200D029E133886B7122E133883C
:1008E0001B0A012B08D10B8812222868934201D8D9
:1008F0000A8892B27E4911E133881B0A022B08D183
:100900000B8843222868934201D80A8892B2794919
:1009100004E133881B0A032B00D007E13388DBB2E4
:10092000012B17D0002B07D0022B00D0FEE00A8845
:100930002868D2B2704911E0042201A86F4900F082
:1009400059FE3B8804222868934201D83A8892B223
:1009500001A9E3E00A8828686949D2B2FFF718FFC5
:10096000E8E03388201C2B71FFF77EFD201CFFF789
:1009700095FDDFE0291C01C90122CFE06149002378
:100980000B8028680222CAE05E4900220A8018888B
:10099000502210405C4A10701E880F203040188092
:1009A0001888032800D9C1E012781B8808335B013E
:1009B000E418A379002A01D09B0600E0DB06DB0FD8
:1009C0000B8028680222A9E019887F2291434E4AB1
:1009D000C9B2117018880F2101401980318800298F
:1009E00000D0A3E01988002900D19FE019880329CD
:1009F00000D99BE012781B8808335B01E318002ABA
:100A000002D020225A718DE0102159718AE00288AB
:100A10007F239A433C4BD2B21A7001880F220A40BE
:100A200002803288002A00D080E00288002A00D1AB
:100A30007CE00288032A00D978E01B78002B1FD0C5
:100A4000038808335B01E3189B799A066AD503880B
:100A5000202208335B01E3181A71038808335B0115
:100A6000E318DB795F065DD50388402208335B011C
:100A7000E318DA710388022208335B01E3181EE0F1
:100A8000038808335B01E3189B79D9064AD50388AC
:100A9000102208335B01E3181A71038808335B01E5
:100AA000E318DB799A063DD50388202208335B01E1
:100AB000E318DA710388012208335B01E3181A7125
:100AC00030E0C046980000207D0000208200002019
:100AD0008400002086000020800000200203000027
:100AE0000103000021200000A121000021220000BC
:100AF0005C160000040000204C1600003C160000AC
:100B0000401600007E0000207C0000200B88082298
:100B10002868934201D80A8892B207490023FFF758
:100B200013FC07E0201CFFF79FFC03E0201C0121C1
:100B3000FFF790FCF7BDC0464800002007B5054B05
:100B40000122019001A91868131CFFF7FDFB012089
:100B50000EBDC0461802002013B5054B6C46073485
:100B60001868211C0122FFF737FC207816BDC0460B
:100B70001802002010B5074C201CFFF711FB031CC6
:100B80000020834205D022684823FF33D05C012334
:100B9000184010BD1802002010B5054A0C1C031C9B
:100BA000191C10680123221CFFF7CEFB201C10BD6E
:100BB0001802002070B5084C061C201C0D1CFFF705
:100BC000EFFA0023984205D02068311C2A1CFFF759
:100BD00003FC031C181C70BD18020020F8B50C4C57
:100BE000051C201C0E1CFFF7DBFA0023271C341CFD
:100BF00098420AD0002C07D0291C221C3868FFF725
:100C0000EBFB241A2D18F5E7331C181CF8BDC04661
:100C10001802002008B5031C081C111C9847044B3F
:100C2000802212055A61034B64221A8008BDC04617
:100C3000004400418C000020012805D1054B064AE4
:100C40001A60064B187004E0002802D1044A014BD8
:100C50001A6070478802002090160000940000205F
:100C6000DC16000030B50A1C1C4985B00978031C4D
:100C700000292AD0042A01D1006804E0022A01D107
:100C8000008800E00078520004A98B180B3B9C1AE6
:100C9000A3420BD00F210140092902D83025294356
:100CA00000E0373119700009013BF1E701A9302359
:100CB0000B7078234B700A208B1898700D20D87019
:100CC000074B04321B68D86803E005490968C86807
:100CD000191CFFF79FFF05B030BDC04688000020FB
:100CE0008802002072B6EFF30883044A1360036899
:100CF00083F30888436818477047C0468C02002079
:100D00000D4B1A88002A09D01A88013A92B21A802B
:100D1000002A03D18022094B12059A61084B1A88D8
:100D2000002A08D01A88013A92B21A80002A02D109
:100D3000044B08221A6070478C00002000440041D8
:100D40008A00002098440041F0B591B008A9CE4A2D
:100D50000B1C31CA31C351CA51C360CA60C3CB4BEB
:100D6000CB489A687A255203520F92005258C949CB
:100D700002609C68A4B262430C60C74900240A6008
:100D8000C64A1460C64C2570C64CC74D2368281C43
:100D90001B6940219847002805D0C44B08221A60DF
:100DA000C34B64221A80C34B00221860C24B1D60E3
:100DB000C24BC24DBF4F1A602A683B689A42E3D2C9
:100DC000BD4B1B681A78FF2A00D120E2232A00D0ED
:100DD000F7E1BB4E3378002B06D0B24BB9491B6804
:100DE0000222D868FFF716FFAD4B1B78532B3FD17B
:100DF0003B682A6893421ED9AF4801322A609A1A8A
:100E0000B14B01681B6801310160B04E9A4201D2BA
:100E1000326000E03360A14832680068049000F05E
:100E2000E9FB336829685A182A60A34A1668F11842
:100E30001160A74A13702B68013B2B609E4B1A6808
:100E4000013A1A60A24BA04A1B7811688B420DD25E
:100E500022689248C91A006892699047002805D014
:100E6000924B08221A60924B64221A80C04696E187
:100E7000522B0ED18948944A2368006811685B6937
:100E800003909847934B802212055A616422924B3B
:100E90000DE04F2B05D1814B8B4A1B6812681A70ED
:100EA0007DE1482B05D17D4B874A1B6812681A806B
:100EB00075E1572B05D1794B834A1B6812681A607C
:100EC0006DE16F2B03D1754B0121186807E0682B8A
:100ED00008D1724B7C481B6802211B880360FFF716
:100EE000C1FE5CE1772B06D16C4B77481B6804216F
:100EF0001B680360F3E7472B13D1734B1868FFF7A8
:100F0000F1FE764B1B6883F3088862B6744B1B783E
:100F1000002B00D143E1634B06201B681B689847F8
:100F20003DE1542B04D1012333705E4B1B6864E018
:100F30004E2B0CD13378002B06D15A4B61491B68DC
:100F40000222D868FFF766FE0023337027E1562B94
:100F500057D123686349D8680122FFF75BFE2368F5
:100F60006149D8680322FFF755FE604D2368291CAC
:100F7000D8680122FFF74EFE23685D49D8680D222C
:100F8000FFF748FE2368291CD8680122FFF742FEBC
:100F9000494F4A4D5749002339602B603A1C281CA1
:100FA00013685E1C16601B780593002B03D0036842
:100FB00001330360F4E73B4E2A683368D868FFF7D3
:100FC00029FE33684949D8680122FFF723FE0599B5
:100FD000296049493960384A1368581C10601B78E9
:100FE000002B04D0354B1A6801321A60F3E73368DE
:100FF0002A68D868FFF70EFE3368D86831490222A4
:10100000CBE0314A582B17D1214E234D3668136857
:101010002A68B10093420AD21C4D5808E86137484B
:1010200028801A4D287DC607FBD55B18F2E71D4BBB
:1010300033491B68D868AFE0592B00D07DE01268B7
:10104000164B3049002A02D11B680B6070E00F4D2F
:10105000086819686B680D4E8025AB439208736071
:10106000002A65D0284B094D2B80084E337DDD07C3
:10107000FBD50023064D2D680195AD08AB4247D343
:10108000224D024E35804AE07016000000400041BB
:101090004002002038020020340200208402002098
:1010A00030020020880200204402002094440041C5
:1010B0008A000020280200202C0200203C02002090
:1010C00088000020D016000090020020940200202A
:1010D00024020020004400418C0000208C020020EB
:1010E00094000020AC160000D5160000AE160000DB
:1010F000F8160000B0160000BC16000002A5FFFFA5
:10110000C51600009000002044A5FFFF04A5FFFFC6
:101110009342B5D09D00465901334E51AAE7404E47
:10112000357DEE07FBD59D0049194019D21A97E786
:101130003C4B3D491B68D8682EE05A2B2FD13B4BC6
:1011400017681D680026EF19BD4206D02878311CAB
:1011500000F014F90135061CF6E7324B34491B68E0
:101160000122D868FFF756FD07230F223240111CD9
:1011700036093031092A00DD07311820C0186A46C7
:101180008154013BF1D2236806A9D8680822FFF7F1
:1011900041FD23682749D8680322FFF73BFD264B12
:1011A0007A221A70254B00221A60254B1B78934235
:1011B0002DD01C4B23491B680122D868FFF72AFD5C
:1011C00025E0111C3039C8B21C4B092804D81D6811
:1011D0002A01114319601AE0111C4139052903D86D
:1011E0001E68373A310106E0111C6139052904D81F
:1011F0001868573A01010A4308E02C2A03D10B4A28
:101200001968116001E00C490A7000221A600E4B47
:101210001A6801321A600D4B1A680132C9E5C046DE
:101220000040004188020020C9160000840200200E
:10123000CD160000CF1600003002002090020020E2
:1012400088000020D31600003C0200202C02002061
:1012500010B51C4B01201A78022402431A701A4B55
:101260000F22197891431970197821431970174981
:101270000C782043087019780A401A701A782021D7
:101280000A431A70124B04211A6A0A431A62114B5C
:10129000114A5A805A7852B2002AFBDBC4220F4806
:1012A0000F499203FEF730FF0E4A002313700E4AD7
:1012B00013700E4A13700E4A13700E4A13700E4AC2
:1012C000137010BD4A440041354400414B44004175
:1012D00000040040000C00401440000000080042E0
:1012E0002AF60000980200201F0300209902002027
:1012F0009C020020200300201D03002008B5C1B27D
:101300000248FEF72FFF012008BDC046000800423A
:10131000024B187E4007C00F7047C04600080042CD
:1013200008B5FFF7F5FF0028FBD00248FEF720FFC5
:1013300008BDC0460008004208B5FFF7E9FF0023DA
:10134000984205D0FFF7ECFF031C233B5A42534160
:10135000181C08BD70B5041C0D1C4618B44204D0FE
:101360002078FFF7CBFF0134F8E7281C70BD10B5DB
:10137000041CFFF7D5FF2070012010BD0B0A584058
:10138000034B4000C05A0902484080B27047C04633
:1013900006170000F7B50024051C0F1C261CBC42D4
:1013A00020D0FFF7BDFF114BC0B21B780190002B7E
:1013B0001AD1311CFFF7E2FF0D4B061C1A88002AD8
:1013C00004D10C4A11782A1C002907D001996A1C03
:1013D0002970802F02D11988013919800134A4B2F3
:1013E000151CDCE7301C00E00120FEBD1D030020C1
:1013F0009A0200201E030020F0B53E4E85B0002268
:1014000003900C1C32703C4B914201D1012201E04F
:101410003A490C801A707F231C4201D080349C43CF
:10142000FFF77EFF3378C0B2002B07D00025357060
:10143000FFF776FF3378C0B2AB4236D1432803D0F2
:10144000712853D01528EBD1012300930120FFF719
:1014500055FF0098FFF752FF00998025C843C0B29E
:10146000FFF74CFF039B00270293244A1388002BAD
:101470001DD1214901930978002918D10198FFF75E
:101480003DFF391C0198FFF779FF013D071C002D36
:10149000EBD1000AC0B2FFF731FFF8B2FFF72EFF21
:1014A000FFF73EFF3378002B0AD035701FE002991A
:1014B000013B09781380029B019101330293DDE720
:1014C000C0B2062807D1009B03990133DBB28031FB
:1014D0000093803C0391002CB8D10420FFF70EFF4D
:1014E000FFF71EFF044B01251C7000E00025281C9F
:1014F00005B0F0BD1D0300201E0300209A0200204D
:10150000F0B5384C87B0002301902370994201D187
:10151000012301E0344A1180344A642613704320C9
:10152000FFF7ECFE324FFFF7F3FE002803D1002F48
:1015300003D0013FF7E7002F03D1013E002EEED18B
:101540004DE00125FFF7ECFE2378002B38D1C0B227
:101550000290012805D004283DD10620FFF7CEFED9
:1015600039E005AE0221301CFFF714FF01988021FD
:10157000FFF710FF23780390002B18D1FFF7D0FE60
:101580000702FFF7CDFEBFB223783F18BFB2012B91
:101590000DD0039B9F4207D13378AB4204D1EB437C
:1015A0007278DBB29A4204D01820FFF7A7FE00231E
:1015B00003E00620FFF7A2FE029B2278002A02D059
:1015C000002626700BE0012B05D1019A6B1C80329E
:1015D000DDB20192B6E7054A002313700126301CE4
:1015E00007B0F0BD1D0300209A0200201E0300205A
:1015F00000350C0010B50023934203D0CC5CC454DA
:101600000133F9E710BD031C8218934202D0197010
:101610000133FAE770470023C25C0133002AFBD193
:10162000581E7047F8B5C046F8BC08BC9E467047C7
:10163000F8B5C046F8BC08BC9E46704704030904D0
:1016400041726475696E6F204C4C43004172647541
:10165000696E6F205A65726F00000000120100026F
:101660000200004041234D00000201020001000081
:1016700008000000100000002000000040000000F2
:1016800080000000000100000002000000040000D3
:10169000FD1200002113000011130000551300007B
:1016A0006F130000F9130000011500007600200000
:1016B00044656320323020323031360031353A33E0
:1016C000363A333900580A0D00590A0D005A0023E2
:1016D0000A0D003E00322E30000000003D0B0000DD
:1016E000590B0000750B0000990B0000B50B0000B2
:1016F000990B0000DD0B00005B41726475696E6F31
:101700003A58595A5D00000021104220633084404D
:10171000A550C660E770088129914AA16BB18CC1C0
:10172000ADD1CEE1EFF13112100273325222B55237
:101730009442F772D662399318837BB35AA3BDD310
:101740009CC3FFF3DEE36224433420040114E66407
:10175000C774A44485546AA54BB528850995EEE560
:10176000CFF5ACC58DD55336722611163006D77617
:10177000F6669556B4465BB77AA719973887DFF7B0
:10178000FEE79DD7BCC7C448E5588668A7784008DF
:10179000611802282338CCC9EDD98EE9AFF9488900
:1017A00069990AA92BB9F55AD44AB77A966A711A77
:1017B000500A333A122AFDDBDCCBBFFB9EEB799B50
:1017C000588B3BBB1AABA66C877CE44CC55C222CC7
:1017D000033C600C411CAEED8FFDECCDCDDD2AADA0
:1017E0000BBD688D499D977EB66ED55EF44E133E57
:1017F000322E511E700E9FFFBEEFDDDFFCCF1BBFF0
:101800003AAF599F788F8891A981CAB1EBA10CD1C9
:101810002DC14EF16FE18010A100C230E3200450D1
:10182000254046706760B9839893FBA3DAB33DC344
:101830001CD37FE35EF3B1029012F322D232354221
:10184000145277625672EAB5CBA5A89589856EF5D4
:101850004FE52CD50DC5E234C324A0148104667471
:10186000476424540544DBA7FAB79987B8975FE724
:101870007EF71DC73CD7D326F2369106B0165766C1
:101880007676154634564CD96DC90EF92FE9C899AC
:10189000E9898AB9ABA94458654806782768C01811
:1018A000E1088238A3287DCB5CDB3FEB1EFBF98B84
:1018B000D89BBBAB9ABB754A545A376A167AF10A61
:1018C000D01AB32A923A2EFD0FED6CDD4DCDAABD94
:1018D0008BADE89DC98D267C076C645C454CA23CB1
:1018E000832CE01CC10C1FEF3EFF5DCF7CDF9BAF64
:1018F000BABFD98FF89F176E367E554E745E932E01
:0C190000B23ED10EF01E000000000000FE
:10190C0001140000090243000201008032090400A6
:10191C00000102020000052400100104240200054D
:10192C00240600010524010001070583030800FFBC
:10193C0009040100020A00000007058102400000B2
:10194C00070502024000000000C201000000080070
:0C195C00690000004100000000000000D5
:0400000300000615DE
:00000001FF
